:020000040000FA
:020000001828BE
:0800080018288207203401349E
:100010000234003404340834083400340834003422
:1000200010340034103400342034003420342034B0
:100030008501860107309F008316A73081001230AA
:1000400085008601831200300520A70061208511FC
:10005000083078200511000085130000051385186D
:100060002F280A30782085182F28051A35280430C3
:10007000A4005820A300031927280517582023029D
:10008000031D2728A40B3E2823080520A7000038BD
:10009000031927282502031D61200F30782005153C
:1000A00014307820851500008513851C55282728D5
:1000B00081016A200108A600113C031CA601260844
:1000C000080085172708A50086040F30782025082A
:1000D000860008003030A000A00B6C280800043017
:1000E000A0005130A100A10B7328A00B71280800BB
:0A00F000A2006F20A20B792808007F
:02400E00103F61
:00000001FF
